:020000040000FA
:100000002E288207003400340034003400341B34BE
:1000100077344034003435346734E03400346A34A3
:10002000CF34C03400349A341D3420340034D534F5
:100030009F34803401341334B234203401344034DA
:100040006F34403401347B34CA3490340134AB34DF
:100050003F3400340134C934C33480348B01073059
:100060009F00BD2383168113FB3085008601831218
:100070000511AD01AE01AF01B001B101E122E122F4
:10008000C220E220D210051A4828D2141D22D21014
:1000900083169B01A5231A088312BB008316A52390
:1000A0001A088312BC008316A5231A088312BD0008
:1000B0008316A5231A088312BE008316A5231A08E7
:1000C0008312A0008316A5231A088312A1008316A9
:1000D000A5231A088312A2008316A5231A088312E7
:1000E000A300FB222923AA22E1220508CB0003302A
:1000F0004B05CA00CC01D0019D21CB198128982045
:100100007C28B501B401B3010130B2004B1A8D282F
:10011000E830B2000330B3008D28CC1891288A2132
:1001200093284D216521FB222923AA22E1227C2844
:10013000CC18A4280430D002D7305007031CA228C2
:100140002830D000B020AB280430D007D73050077B
:100150000318D001B020FB222923AA22E1220800A3
:1001600050080120A300D00A50080120A200D00AA4
:1001700050080120A100D00A50080120A00003303F
:10018000D0020800B423033086000616B4230612FA
:10019000033086000616B7230612033086000616C3
:1001A000B7230612023086000616BA23061228303C
:1001B00076230830762301307623063076230C3000
:1001C000762308008030762350307A2349307A2312
:1001D00043307A2345307A234C307A2367307A23B0
:1001E00065307A236E307A238830C3007623373027
:1001F0007A232E307A2331307A232D307A23363009
:100200007A2330307A2320307A2320307A23C0308A
:10021000762350307A2349307A2343307A2347308B
:100220007A2345307A234E307A2320307A233730B0
:100230007A232E307A2331307A2320307A232030EB
:100240007A2320307A2320307A2320307A232030FA
:100250007A23A923C030762320307A2320307A23D2
:1002600020307A2320307A2320307A2320307A23DA
:1002700020307A2320307A2320307A2320307A23CA
:1002800020307A2320307A2320307A2320307A23BA
:1002900020307A2320307A2308003208A007031C7C
:1002A0005629A10F5629A20F5629A30A3308A107E0
:1002B000031C5D29A20F5D29A30A3408A207031CB1
:1002C0006229A30A3508A3070800FC302307031896
:1002D000812903302302031C89296C30220703186B
:1002E000812993302202031C8929783021070318C1
:1002F000812987302102031C892900302002031C38
:1003000089290030A0008730A1009330A20003307B
:10031000A3000800B209B309B409B509B20F9529C1
:10032000B30F9529B40F9529B50A4D21A31F9C2918
:10033000A001A101A201A3010800D21CCB21050844
:10034000CB00BF2305084B06031D9D2903304B0539
:10035000C9004A0603199D290310CA0D4908CA0697
:100360004A080239CD004C06CC01CA18BF294908F9
:10037000CA00CF034F189D29CF189D29C8290230E4
:10038000CC004908CA00CF0A4F189D29CF189D29D3
:100390004908CA000800051ED0298519D929D52980
:1003A0008519D7295218DB29EE2952141C2A52101C
:1003B0001C2AD2011C2A1030D300051AE429B123CB
:1003C000D30BDD2991221C2AB5010F30B400423035
:1003D000B3004030B2004D216521182A1030D300FF
:1003E0008519102AB123D30BF0299122CB30762323
:1003F00053307A2341307A2356307A2345307A239A
:1004000044307A23A923CB30762320307A2320303E
:100410007A2320307A2320307A2320307A231C2A32
:10042000B5010F30B4004230B3004030B2008A2131
:10043000FB222923AA22E12208008030A000963066
:10044000A1009830A2000030A30083169B01A523D1
:100450001A088312BB008316A5231A088312BC0056
:100460008316A5231A088312BD008316A5231A0834
:100470008312BE00FB222923C430C30076234330FD
:10048000C3007A234130C3007A234C30C3007A235F
:10049000AA22E1229D21B501B401B3011030B200BE
:1004A0004B19542A8030B2000000CC18622AB209DD
:1004B000B309B409B509B20F622AB30F622AB40FA7
:1004C000622AB50A3208BB07031C6B2ABC0F6B2AD1
:1004D000BD0F6B2ABE0A3308BC07031C722ABD0F6E
:1004E000722ABE0A3408BD07031C772ABE0A3508E3
:1004F000BE07051E482A3B0883169B019A009823D5
:1005000083123C0883169A00982383123D088316B1
:100510009A00982383123E0883169A009823831228
:100520000800831604309B008312200883169A006B
:1005300098238312210883169A0098238312220895
:1005400083169A0098238312230883169A0098230F
:1005500083120800AD01AE01AF01B001B10120303E
:10056000B8003B08BF003C08C0003D08C1003E0881
:10057000C20003103F1CD32A2008AE07031CC52A63
:10058000AF0FC52AB00FC52AB10A2108AF07031C57
:10059000CC2AB00FCC2AB10A2208B007031CD12AFA
:1005A000B10A2308B107B10CB00CAF0CAE0CAD0C06
:1005B000C20CC10CC00CBF0CB80BB92A0130B10081
:1005C00008002D3084000008BA000830B900BA0CC9
:1005D000031CEE2A861506150611F12A861106154A
:1005E0000611B90BE72A840A32300402031CE32AFD
:1005F0008617861308002030B600A801A901AA01B9
:10060000AB01AC010310A00DA10DA20DA30D0318A9
:100610002014A80DA90DAA0DAB0DAC0DB603031D3A
:10062000122B0800283084001E23840A1E23840A0B
:100630001E23840A1E23840A1E23022B0330000774
:10064000B700B719800030300007B700B71B800033
:1006500008008030762320307A232B0E0F39303E6D
:100660007A232B080F39303E7A232C307A232A0E36
:100670000F39303E7A232A080F39303E7A23290E6B
:100680000F39303E7A232E307A238830762329089A
:100690000F39303E7A23280E0F39303E7A2328084E
:1006A0000F39303E7A2320307A236B307A2348305A
:1006B0007A237A307A2320307A2308008601831641
:1006C00008308600831206138616FF30C500061612
:1006D0000608C400061200000000061600000612FC
:1006E000C5030319752BC419672B0800C300D1017A
:1006F00006137D2BC300511406175E238601831653
:100700000030860083128612061351180617F03047
:100710008605430E0F398604061600000612F030D7
:10072000860543080F3986040616000006120800E5
:100730001C158B1355309D00AA309D009C149C18ED
:100740009F2B9C171C119B0A08001C141A089B0A5B
:100750000800AE23AE23AE23AE230800B123B1239D
:100760000800FF30C500C12B8030C500C12B4030D0
:10077000C500C12B2030C500C12B1030C500023090
:10078000C500FF30C600C60BC32BC50BC12B08002C
:02400E00303F41
:10420000DE006500DC00170028000100D600000079
:10421000000000000000000000000000000000009E
:10422000000000000000000000000000000000008E
:10423000000000000000000000000000000000007E
:10424000000000000000000000000000000000006E
:10425000000000000000000000000000000000005E
:10426000000000000000000000000000000000004E
:10427000000000000000000000000000000000003E
:10428000000000000000000000000000000000002E
:10429000000000000000000000000000000000001E
:1042A000000000000000000000000000000000000E
:1042B00000000000000000000000000000000000FE
:1042C00000000000000000000000000000000000EE
:1042D00000000000000000000000000000000000DE
:1042E00000000000000000000000000000000000CE
:00000001FF
